:100000000C947C020C94C0020C94C0020C94C002AC
:100010000C94C0020C94C0020C94C0020C94C00258
:100020000C94C0020C94C0020C94AC0D0C947E0E87
:100030000C94C0020C94C0020C94C0020C94C00238
:100040000C94C0020C9488220C94C0020C94C00240
:100050000C94C0020C941B1C0C94C0020C94C002A3
:100060000C94C0020C94C0020C94C0020C94C00208
:100070000C94C0020C94C0020C94C0020C94C002F8
:100080000C94C0020C94C0020C94C0020C94C002E8
:100090000C94C0020C94C0020C94C0020C94C002D8
:1000A0000C94C0020C94C0020C94C002EB0E0D0F15
:1000B000FB0F0D0FFB0F520F750FFB0FCA0FDD0F5C
:1000C000AC12AC12DB12DB12111331136214621486
:1000D0003C136214EC13EC135314621462145C149A
:1000E000F913F913F913F913F913F913F913F913B0
:1000F000F913F913F913F913F913F913F913F913A0
:100100000B1418141F14261430140000F0A100C89A
:1001100001C82E004C002A008450354100001E000A
:10012000140004001D7134004D001F001A00160059
:100130001B00E104145020000800070006005000D6
:100140002C0021001500090019004F004A00220070
:1001500017000A00050000006574500001540000FB
:100160002F7F0000E3004F000154000030770000B3
:10017000E20023001C000B00110000002971240084
:1001800018000D74100052004B0025000C000E00EA
:10019000360051002800260012000F0037002F0003
:1001A0002B41270013003342387130004E002D00E0
:1001B0003100347885502D4100000100010001001C
:1001C0000100010000003A0001001E0023000100B0
:1001D00001003B0001001F002400010001003C0061
:1001E0000100200025004B0101003D00010021001D
:1001F00026004E0101003E00010022002700000001
:1002000001000100010000000100000001000100E8
:10021000010000000100000001003F000100240275
:10022000310200000100400001002D021F02010008
:100230000100410001002D002E00010001004200DC
:1002400001001300220201000100430001002E0200
:10025000010001000100440045000100010001000F
:100260000000010001000100010001000000010088
:1002700001004B00010001000100010001004A00E3
:10028000010001000100010001004D00010001001A
:100290000100010001004E00010001000100010009
:1002A0000100010001000000010001000100000048
:1002B0000100000001000100010000000100000039
:1002C0000100010001000100010000000100010027
:1002D000010001000100A90001000100010001006E
:1002E000AC00AA00B600010001000100AB00A800AC
:1002F00001000100010001000100010001000100F6
:100300000100AE000100010000001603450072006C
:1003100067006F0044006F007800200045005A001D
:10032000000016034500720067006F0044006F0074
:100330007800200045005A00000004030904090267
:100340006D00040100A0FA0904000001030101008E
:10035000092111010001223F000705810308000A5D
:100360000904010001030102000921110100012219
:100370004D000705820308000A090402000103007A
:10038000000009211101000122360007058303083E
:10039000000A090403000103000000092111010003
:1003A0000122390007058403100001120110010029
:1003B000000008EDFE07130100010200010501091C
:1003C00006A101050719E029E71500250195087523
:1003D000018102050819012905950575019102950C
:1003E000017503910105071900297715002501956D
:1003F0007875018102C005010980A10185021601FD
:100400000026B7001A01002AB70075109501810077
:10041000C0050C0901A1018503160100269C021AE2
:1004200001002A9C02751095018100C00501090296
:10043000A1010901A10005091901290515002501DE
:10044000950575018102950175038101050109304A
:1004500009311581257F95027508810609381581B6
:10046000257F950175088106050C0A38021581253E
:100470007F950175088106C0C005010906A1010527
:100480000719E029E71500250195087501810295F6
:100490000175088101050819012905950575019166
:1004A000029501750391010507190029FF15002523
:1004B000FF950675088100C00000000000000000E4
:1004C000000000010204060A0F17202C3A4A5D7151
:1004D000879DB3C7DAE9F5FCFFFCF5E9DAC7B39D00
:1004E00087715D4A3A2C20170F0A060402010000AA
:1004F000000000000000000011241FBECFEFDAE072
:10050000DEBFCDBF04B603FE24C08091FB019091F5
:10051000FC01A091FD01B091FE018730904BA740F6
:10052000B04BB9F41092FB011092FC011092FD0146
:100530001092FE0114BE84B7877F84BF88E10FB696
:10054000F89480936000109260000FBEE0E0FFE33B
:10055000099511E0A0E0B1E0EEE9F8E402C00590F1
:100560000D92A433B107D9F711E0A4E3B1E001C0C3
:100570001D92AB3FB107E1F70E94F00A0C944D24A5
:100580000C9400001092B9008AE08093B80008959E
:1005900094EA9093BC009091BC0097FFFCCF90919F
:1005A000B900987F983021F0903111F081E00895E2
:1005B0008093BB0084E88093BC008091BC0087FFDF
:1005C000FCCF8091B900887F883111F0803471F7B9
:1005D00080E0089584E98093BC008091BC0084FD94
:1005E000FCCF08958093BB0084E88093BC00809189
:1005F000BC0087FFFCCF9091B900987F81E09832D2
:1006000009F480E0089584E88093BC008091BC00E8
:1006100087FFFCCF8091BB0008958091010181117B
:1006200015C080E40E94C8028093010181110CC0B2
:1006300082E10E94F20280930101811105C08FEFD7
:100640000E94F202809301010E94EA0284B1807F3D
:1006500084B985B1807F85B98AB1837F8AB98BB12E
:10066000837F8BB93E98469808950E94C804809372
:1006700001010E940D0380B38C7080BB81B3836F36
:1006800081BBA5E3B1E0E3E4F1E08EE08E0F1192CF
:100690001D928E13FCCF0C94B204BF92CF92DF92C6
:1006A000EF92FF920F931F93CF93DF9380910101FD
:1006B000882379F0809134018F5F80933401811118
:1006C00008C00E94C80480930101811102C00E94E9
:1006D0005A0405E311E0C0E0D0E0DD24D39482E0C9
:1006E000C82EEE24E394F12CC730D10500F580919B
:1006F0000101811164C080E40E94C802809301015D
:10070000811112C082E10E94F202809301018111E5
:100710000BC0C7010C2E01C0880F0A94EAF7809520
:100720000E94F202809301010E94EA0248C0CA308E
:10073000A1F028F4C83059F0C93061F005C0CC30C0
:1007400089F070F0CD3089F0209A289810C0219A55
:1007500029980DC0229A2A980AC0239A2B9807C07C
:10076000529A01C0539A5B9802C03E9A469890EA0A
:100770009A95F1F79FB1799902C082E001C080E0BB
:1007800091709D25982B7C9902C084E001C080E087
:10079000892B7D9902C038E001C030E0832B7E991F
:1007A00002C020E101C020E0822B9FB19095991FEB
:1007B0009927991F9295990F907E892B0FC0809150
:1007C0000101811149C080E40E94C80280930101A7
:1007D000882379F1B12C0E94EA028B2DF8019081D7
:1007E000981719F08083C09200010E940D03219692
:1007F0000F5F1F4FCE30D10509F076CF80910001F9
:10080000882361F1815080930001882339F08FE9BA
:100810009FE00197F1F700C0000020C0A3E4B1E021
:10082000E5E3F1E0CF01825F91919D938E13FCCFC0
:1008300015C083E10E94F202809301018111CACFA9
:1008400081E40E94C802809301018111C3CF0E94FC
:100850000303B82EB094BFCF80E0C0CF0E945804ED
:1008600081E0DF91CF911F910F91FF90EF90DF908A
:10087000CF90BF900895E82FF0E0ED5BFE4F8081B0
:10088000089508950F931F93CF93DF93C3E4D1E0AE
:1008900010E00C2F025F899190E00E94411B180F1D
:1008A0000C13F9CF812FDF91CF911F910F910895F4
:1008B0000C941B0556985E9825982D9826982E988E
:1008C00027982F988FEF90E090938900809388006D
:1008D00090938B0080938A0090938D0080938C007E
:1008E000259A2D9A2FEF80E792E02150804090408A
:1008F000E1F700C00000269A2E9A2FEF80E792E0E1
:10090000215080409040E1F700C00000279A2F9AC4
:100910002FEF80E792E0215080409040E1F700C047
:10092000000025982D982FEF80E792E0215080401D
:100930009040E1F700C0000026982E982FEF80E746
:1009400092E0215080409040E1F700C000002798DD
:100950002F9856985E9825982D9826982E98279827
:100960002F98089589EA8093800089E08093810020
:1009700024982C983F988AB18F748AB96E98479AB8
:100980008BB1806B8BB9769A0E945A040C941A052D
:1009900080E2809301018091510181110EC00E947B
:1009A000C20281E0809351012FEF83ED90E321504B
:1009B00080409040E1F700C0000080E40E94C8023F
:1009C0008093010181112EC00E94F20280930101E7
:1009D000811128C00E94F20280930101811122C07E
:1009E0008FE30E94F2028093010181111BC00E94DB
:1009F000EA0280E40E94C80280930101811112C0C2
:100A00008CE00E94F2028093010181110BC00E94D0
:100A1000F20280930101811105C08FE30E94F2026E
:100A2000809301010E94EA0280910101089580E013
:100A300090E0089508956091BD017091BE0180918C
:100A4000BF019091C0010E944D1B56985E98259859
:100A50002D9826982E9827982F98813029F082304B
:100A600029F4269A2E9A02C0259A2D9A80915D012A
:100A7000882309F450C080915B0190915C010E9431
:100A8000F11B8D3291400CF446C010925D010E9422
:100A9000930580915501909156014A97C1F4809138
:100AA000570190915801892B91F4809159019091AF
:100AB0005A01892B61F482EE0E9450118DE30E944D
:100AC00050118DE30E94181282EE0E94181280913C
:100AD0005501909156014297F1F480915701909100
:100AE0005801892BC1F48091590190915A01892BA9
:100AF00091F480EE0E94501181EE0E94501182E12B
:100B00000E94501182E10E94181281EE0E94181278
:100B100080EE0C941812089581E0089581E0089504
:100B20000C948E05089508950F931F93CF93DF9330
:100B30008C01FC01C081D181CE010E94C619BE0189
:100B40000E943D06EC01B8010E949005882309F43B
:100B50008DC0F8018281882309F44AC080915D012B
:100B600081111FC0C431F0E5DF0709F051C00E94B8
:100B7000920581E080935D010E94E51B90935C01EA
:100B800080935B011092540110925601109255010E
:100B9000109258011092570110925A011092590167
:100BA00065C080915B0190915C010E94F11B883CC3
:100BB000910570F480915401E82FF0E0EE0FFF1FD3
:100BC000EB5AFE4FD183C0838F5F809354014EC098
:100BD000C43880E5D80721F0C538D04501F13AC0C6
:100BE000F8018281882341F01092520182E01EC0F8
:100BF000C438E0E5DE0759F580915201811106C045
:100C000086E20E94501186E20E94181282E01CC007
:100C1000C438F0E5DF0741F3C538D045D9F4F80111
:100C20008281882331F01092530180E20E94671282
:100C30001DC080915301811106C087E20E945011AE
:100C400087E20E94181280E20E946E120FC0C5381F
:100C5000D04529F381E08093520180935301C8016C
:100C6000DF91CF911F910F910C948C0580E0DF9163
:100C7000CF911F910F910895089596E0799FF0010B
:100C8000112494E5899FE00DF11D1124E60FF11D5B
:100C9000EE0FFF1FEE5EFE4F859194910895880F31
:100CA000991FFC01E657F040859194910895880FB3
:100CB000991FFC01E65FFE4F8591949108950F9373
:100CC0001F93CF93DF93EC01811520E3920750F53A
:100CD000C11580E2D80708F0C3C0CB3BD10590F422
:100CE000C83AD10508F06AC0C53AD10508F05BC022
:100CF000C430D10508F0D0C1219709F0CAC101E084
:100D000010E00AC2CF3FD10511F008F0C5C1C03FC5
:100D1000D10508F0A2C0CE01805E9109089708F4C1
:100D2000BBC1B7C1C13090E5D90709F4A2C020F515
:100D3000C0318FE4D80770F4C11590E4D90708F0EA
:100D400094C0C11521E3D20708F0A3C1DD278E01AD
:100D5000106CE2C1C115D04509F09BC10E94CD14B1
:100D60008FEF94E32CE0815090402040E1F700C0E9
:100D700000000E94401CD0C1C11597E5D90758F466
:100D8000C03121E5D20708F01CC1C43180E5D80785
:100D900008F475C07EC1CE0190578115904108F0CE
:100DA00078C1DF7073C1C53AD10509F477C1C63A7D
:100DB000D10509F076C102E810E4AEC1C83AD10508
:100DC00009F472C1C93AD10509F471C1CA3AD10511
:100DD00009F470C1CB3AD10509F46FC1CC3AD10501
:100DE00009F46EC1CD3AD10509F46DC1C03BD105FE
:100DF00009F46CC1CE3AD10509F46BC1CF3AD105E3
:100E000009F46AC1C13BD10509F469C1C23BD105EE
:100E100009F468C1C33BD10509F467C1C43BD105DE
:100E200009F466C1C53BD10509F465C1C63BD105CE
:100E300009F464C1C73BD10509F463C1C83BD105BE
:100E400009F462C1C93BD10509F461C1CA3BD105AE
:100E500009F460C100E014E45FC18E0110655CC15B
:100E6000CE019F700E94570658C1DF708E01106A34
:100E700053C18091DA0181608093DA014DC10E94F3
:100E8000E51D811102C00E94CB1D0E94021E90E050
:100E90009093FB018093FA01C23080E5D80721F4DA
:100EA0008091FA01816086C0C43090E5D90721F4B1
:100EB0008091FA0182607EC0C63020E5D20721F41D
:100EC0008091FA01846076C0C83080E5D80719F4B3
:100ED0008091FA0127C0CA3090E5D90721F48091AA
:100EE000FA01806167C0CC3020E5D20721F48091FF
:100EF000FA0180625FC0CE3080E5D80721F480918E
:100F0000FA01806457C0C03190E5D90721F480917F
:100F1000FA0180684FC0C23120E5D20729F48091E0
:100F2000FA018460886046C0C33080E5D80721F4A8
:100F30008091FA018E7F3EC0C53090E5D90721F43B
:100F40008091FA018D7F36C0C73020E5D20721F4A9
:100F50008091FA018B7F2EC0C93080E5D80719F443
:100F60008091FA0126C0CB3090E5D90721F4809119
:100F7000FA018F7E1FC0CD3020E5D20721F4809189
:100F8000FA018F7D17C0CF3080E5D80721F480911A
:100F9000FA018F7B0FC0C13190E5D90721F4809110
:100FA000FA018F7707C0C331D04531F48091FA013F
:100FB0008B7F877F8093FA018091FA010E94061E41
:100FC000ABC08D2F99278F70992781309105D9F467
:100FD0009E012370332702C0880F991F2A95E2F7DC
:100FE0009C688E0144E0000F111F4A95E1F700272D
:100FF0001370802B912B53E0CC0FDD1F5A95E1F736
:10100000C076DD272FC08230910531F4DC2FCC274C
:101010008E01016F106A80C08330910569F4CE01A2
:101020008370992701E010E002C0000F111F8A951C
:10103000E2F7C8019C680FC084309105B9F4CE0175
:101040008370992701E010E002C0000F111F8A95FC
:10105000E2F7C8019A6823E0CC0FDD1F2A95E1F77B
:10106000C07ED7708C010C2B1D2B56C0853091058E
:1010700031F4DC2FCC278E01046F106A4DC0069727
:1010800009F04AC0CF71DD27DC2FCC278E0110621A
:1010900043C000E010E040C08E013EC001E810E413
:1010A0003BC003E810E438C002EE14E435C009EE9A
:1010B00014E432C00AEE14E42FC005EB14E42CC093
:1010C00006EB14E429C007EB14E426C00CEC14E48E
:1010D00023C00DEC14E420C003E815E41DC00AE8A9
:1010E00015E41AC002E915E417C004E915E414C0B8
:1010F00001E216E411C003E216E40EC004E216E4B5
:101100000BC005E216E408C006E216E405C007E2DB
:1011100016E402C00AE216E4C801DF91CF911F91E4
:101120000F91089596E0799FF001112494E5899F2D
:10113000E00DF11D1124E60FF11DEE0FFF1FEE5E15
:10114000FE4F85919491803E9105E0F4803C91059D
:1011500058F58133910509F46FC048F4893291053F
:1011600009F463C08A32910509F46DC072C08933F5
:101170009105E9F082389105D1F08533910509F4A4
:101180004DC067C0833E910581F138F4803E9105E2
:10119000B9F0823E9105D9F05CC0863E910561F1BF
:1011A000873E9105A1F155C00E944F0608952091F8
:1011B000FA0120FD02C021FF4CC080EE90E049C042
:1011C0008091FA0180FFF9CF89E390E042C08091DD
:1011D000FA0182FF0EC08091FA0184FF03C080E013
:1011E00090E037C083EE90E034C08091FA0182FF36
:1011F000F2CF82EE90E02DC08091FA0183FF0BC008
:101200008091FA0184FDEBCF87EE90E022C08091BF
:10121000FA0183FFF5CF86EE90E01BC08091FA01C2
:1012200085FF07C089E290E014C08091FA0185FF34
:10123000F9CF85E390E00DC08091FA0186FF07C0E9
:101240008AE290E006C08091FA0186FFF9CF81E33F
:1012500090E00E945F06089508950C942C098091F7
:101260006E010895CF93DF9300D01F92CDB7DEB704
:101270009C018091F101843019F593E099833B83BF
:101280002A839093E9008FEF9091E800815095FDBB
:1012900006C095ED9A95F1F700008111F5CF809188
:1012A000E80085FF0DC040E050E063E070E0CE0153
:1012B00001960E949C0B8091E8008E778093E80055
:1012C0000F900F900F90DF91CF910895CF93DF9300
:1012D00000D01F92CDB7DEB72091F101243021F567
:1012E00022E029839B838A8383E08093E9008FEF48
:1012F0009091E800815095FD06C095ED9A95F1F723
:1013000000008111F5CF8091E80085FF0DC040E01D
:1013100050E063E070E0CE0101960E949C0B80914A
:10132000E8008E778093E8000F900F900F90DF9188
:10133000CF9108952091F1012430F1F422E020931F
:10134000E9002FEF3091E800215035FD06C035ED62
:101350003A95F1F700002111F5CF2091E80025FF23
:101360000BC040E050E065E070E00E949C0B809173
:10137000E8008E778093E8000895CF93DF93EC0127
:101380009091F101943009F046C080910C018823BE
:10139000D9F080910D018823B9F09093E9008FEF87
:1013A0009091E800815095FD06C095E19A95F1F77E
:1013B00000008111F5CF8091E80085FF2CC040E04E
:1013C00050E060E170E017C081E08093E9008FEFAA
:1013D0009091E800815095FD06C095ED9A95F1F742
:1013E00000008111F5CF8091E80085FF14C040E036
:1013F00050E068E070E0CE010E949C0B8091E80014
:101400008E778093E80080E1FE01AEE5B1E00190C7
:101410000D928A95E1F7DF91CF9108958091F001C7
:10142000811109C00E94310D0E948E0D8091E20051
:1014300084608093E20008951092F0010895089569
:101440000C9475220E94D61B0E947B220E943410AD
:101450000C942D0942E061EC81E00E94AB0C42E06B
:1014600061EC82E00E94AB0C42E061EC83E00E9400
:10147000AB0C42E161EC84E00C94AB0C8091F30185
:10148000833009F455C030F4813071F0823009F4B2
:101490008EC008958A3009F47AC08B3009F460C098
:1014A000893009F09CC020C08091F201813A09F096
:1014B00096C08091E800877F8093E8008091F601D4
:1014C0009091F701892B21F460E18EE591E003C052
:1014D00060E080E090E070E00E94E70B8091E8001F
:1014E0008B778093E80008958091F201813209F0B2
:1014F00076C08091F6019091F701009719F003975B
:1015000009F06DC08091E800877F8093E8008091AA
:10151000E80082FD05C08091F1018111F8CF5FC024
:101520008091F10080936E018091E8008B7753C029
:101530008091F201813A09F052C08091F6019091B8
:10154000F701892B09F04BC08091E800877F8093D9
:10155000E8008091E80080FFFCCF80910C0136C04C
:101560008091F2018132D9F58091F6019091F701D5
:10157000892BA9F58091E800877F8093E8000E947D
:10158000E00C8091F40180930C010C94CD148091B7
:10159000F201813221F58091E800877F8093E80095
:1015A0000E94E00C8091F50180936F010895809175
:1015B000F201813AA1F48091E800877F8093E800EE
:1015C0008091E80080FFFCCF80916F018093F10053
:1015D0008091E8008E778093E8000C94E00C0895E9
:1015E00084B7877F84BF88E10FB6F894809360004A
:1015F000109260000FBE90E080E80FB6F8948093E0
:101600006100909361000FBE0E9483100E94310D13
:101610000E948E0D8091E20084608093E2007894B5
:101620000E9414100E94851082E091E00E942F1009
:101630000E9463228091F101853069F40E949D1B14
:101640008091EF018823B1F30E94C81B882391F396
:101650000E94860BEFCF0E948B10ECCF292F3327EF
:1016600023303105C9F064F42130310581F0223096
:10167000310509F043C08DE690E02EE333E042C02F
:1016800021323105F1F02232310541F137C082E1DA
:1016900090E02BEA33E036C099278130910541F084
:1016A0008230910541F0892B49F5EAE3F3E005C06A
:1016B000E2E2F3E002C0EAE0F3E0849190E09F010F
:1016C00021C06430D8F4E62FF0E0EE0FFF1FEE5D8E
:1016D000FE4F2081318189E090E014C0643070F4C5
:1016E00070E0FB01EE0FFF1FE65EFE4F20813181AF
:1016F000FB01EA5EFE4F808190E004C080E090E054
:1017000020E030E0FA0131832083089580E189BD33
:1017100082E189BD09B400FEFDCF8091D8008F7DA4
:101720008093D8008091E00082608093E0008091F7
:10173000E00081FDFCCF0895CF92DF92EF92FF92FF
:101740000F931F93CF93DF93EC018B016A010E94EB
:10175000FF0C811133C0C114D10439F0F60180812E
:101760009181081B190BC80FD91FE12CF12C011511
:10177000110519F18091E80085FD16C08091E800FF
:101780008E778093E800C114D10449F0F60180817E
:101790009181E80EF91EF182E08285E00FC00E947F
:1017A000FF0C882321F30AC089918093F100015036
:1017B0001109FFEFEF1AFF0ADACF80E0DF91CF9136
:1017C0001F910F91FF90EF90DF90CF90089520919F
:1017D000F8013091F9012617370748F061157105B6
:1017E00039F42091E8002E772093E80001C0B90178
:1017F00040E061157105A9F12091F101222309F45E
:1018000043C0253009F442C02091E80023FD40C0C8
:101810002091E80022FD32C02091E80020FFE9CFAE
:101820004091F3002091F20030E0342BFC01CF0115
:101830006115710559F02830310540F4819180938C
:10184000F100615071092F5F3F4FF1CF41E0283027
:10185000310509F040E02091E8002E772093E80060
:10186000C8CF4111C9CF0AC08091F101882361F02E
:10187000853061F08091E80083FD0AC08091E80026
:1018800082FFF2CF80E0089582E0089583E008951A
:1018900081E008952091F8013091F901261737076A
:1018A00048F06115710539F42091E8002E772093F6
:1018B000E80001C0B901FC0120E06115710591F15A
:1018C0008091F101882309F440C0853009F43FC0BC
:1018D0008091E80083FD3DC08091E80082FD2FC02B
:1018E0008091E80080FFE9CF2091F3008091F20021
:1018F00090E0922B6115710559F08830910540F404
:1019000024912093F1003196615071090196F2CF34
:1019100021E0089709F020E08091E8008E7780931D
:10192000E800CBCF2111CCCF0AC08091F1018823F0
:1019300061F0853061F08091E80083FD0AC08091FC
:10194000E80082FFF2CF80E0089582E0089583E00E
:10195000089581E00895982F973058F59093E90005
:10196000981739F07091EC002091ED005091F00043
:1019700003C0242F762F50E021FF19C03091EB00D7
:101980003E7F3093EB003091ED003D7F3093ED00D2
:101990003091EB0031603093EB007093EC002093BA
:1019A000ED005093F0002091EE0027FF07C09F5FED
:1019B000D3CF8F708093E90081E0089580E008958F
:1019C0008091F20187FF11C08091E80082FD05C07F
:1019D0008091F1018111F8CF11C08091E8008B77DF
:1019E0000BC08091F101882349F08091E80080FFCD
:1019F000F8CF8091E8008E778093E80008952091D9
:101A0000E4003091E50095E64091EC00842F817070
:101A100040FF22C08091E80080FD1CC08091F10150
:101A2000882391F0853091F08091EB0085FD10C006
:101A30004091E4005091E5004217530729F39A01C1
:101A4000915011F784E0089582E0089583E00895AD
:101A500081E0089580E008954091E80042FFDECFE4
:101A600008950E949F0D0E94A70DE0EEF0E0808196
:101A700081608083E8EDF0E080818F77808319BCFE
:101A8000A7EDB0E08C918E7F8C9380818F7E8083D8
:101A90001092F00108950F931F93CF93DF930E944C
:101AA0009F0D0E94A70DC8EDD0E088818F778883B5
:101AB00088818068888388818F7D888319BC109293
:101AC000F1011092ED011092EF011092EE0100EE83
:101AD00010E0F80180818B7F80838881816088831A
:101AE00042E060E080E00E94AB0CE1EEF0E080813B
:101AF0008E7F8083E2EEF0E0808181608083808150
:101B000088608083F80180818E7F808388818061F6
:101B10008883DF91CF911F910F910895E8EDF0E058
:101B200080818F7E8083E7EDF0E08081816080831B
:101B300084E082BF81E08093F0010C944B0DE8EDCE
:101B4000F0E080818E7F80831092E20008951092F1
:101B5000DA001092E10008951F920F920FB60F92D3
:101B600011242F933F934F935F936F937F938F93A2
:101B70009F93AF93BF93EF93FF938091E10082FF18
:101B80000BC08091E20082FF07C08091E1008B7F53
:101B90008093E1000E9413108091DA0080FF1FC043
:101BA0008091D80080FF1BC08091DA008E7F8093E7
:101BB000DA008091D90080FF0DC080E189BD82E10B
:101BC00089BD09B400FEFDCF81E08093F1010E9440
:101BD0000E0A05C019BC1092F1010E941C0A8091E6
:101BE000E10080FF19C08091E20080FF15C0809164
:101BF000E2008E7F8093E2008091E200806180931A
:101C0000E2008091D80080628093D80019BC85E002
:101C10008093F1010E94200A8091E10084FF30C08E
:101C20008091E20084FF2CC080E189BD82E189BD02
:101C300009B400FEFDCF8091D8008F7D8093D8003D
:101C40008091E1008F7E8093E1008091E2008F7EA1
:101C50008093E2008091E20081608093E2008091B5
:101C6000ED01882311F084E007C08091E30087FD37
:101C700002C081E001C083E08093F1010E94220A4A
:101C80008091E10083FF29C08091E20083FF25C09D
:101C90008091E100877F8093E10082E08093F101F1
:101CA0001092ED018091E1008E7F8093E1008091A0
:101CB000E2008E7F8093E2008091E2008061809359
:101CC000E20042E060E080E00E94AB0C8091F00016
:101CD00088608093F0000E941F0AFF91EF91BF91EE
:101CE000AF919F918F917F916F915F914F913F91B4
:101CF0002F910F900FBE0F901F9018951F920F926B
:101D00000FB60F9211242F933F934F935F936F93CE
:101D10007F938F939F93AF93BF93CF93DF93EF9373
:101D2000FF93C091E900CF708091EC00D82FD17063
:101D300080FDD0E81092E9008091F000877F8093C9
:101D4000F00078940E94C20E1092E9008091F00099
:101D500088608093F000CD2BCF70C093E900FF9195
:101D6000EF91DF91CF91BF91AF919F918F917F9133
:101D70006F915F914F913F912F910F900FBE0F90F8
:101D80001F9018951F93CF93DF93CDB7DEB7AA9717
:101D90000FB6F894DEBF0FBECDBFE2EFF1E088E0F2
:101DA0008E0F9091F10091938E13FBCF0E943E0A0B
:101DB0008091E80083FF1FC18091F2019091F301AF
:101DC000492F50E04A30510508F015C1FA01EA5A8E
:101DD000FF4F0C94FD23803881F0823809F00BC14D
:101DE0008091F6018F708093E9008091EB0085FB74
:101DF000882780F91092E90006C08091EE01909149
:101E0000EF01911182609091E800977F9093E80034
:101E10008093F1001092F100C8C0282F2D7F09F0A7
:101E2000EAC0882319F0823061F0E5C08091F401A6
:101E3000813009F0E0C0933009F080E08093EF0139
:101E40002BC08091F401811127C08091F6018F7021
:101E500009F4D1C08093E9002091EB0020FF1CC061
:101E6000933021F48091EB00806214C09091EB00DC
:101E700090619093EB0021E030E0A90102C0440F93
:101E8000551F8A95E2F74093EA001092EA0080918C
:101E9000EB0088608093EB001092E9008091E800ED
:101EA000877F86C08111A7C01091F4011F778091B0
:101EB000E3008078812B8093E3008091E800877FA6
:101EC0008093E8000E94E00C8091E80080FFFCCF46
:101ED0008091E30080688093E300111102C082E0EA
:101EE00001C083E08093F10186C08058823008F001
:101EF00082C08091F4019091F5018C3D53E09507EB
:101F000079F583E08A838AE289834FB7F894DE010A
:101F1000139620E03EE051E2E32FF0E050935700AB
:101F2000E49120FF03C0E295EF703F5FEF708E2FCA
:101F300090E0EA3010F0C79601C0C0968D939D9353
:101F40002F5F243149F74FBF8091E800877F80934E
:101F5000E8006AE270E0CE0101960E94E70B14C02F
:101F6000AE014F5F5F4F6091F6010E942E0BBC01E6
:101F7000009709F440C09091E800977F9093E800A3
:101F800089819A810E944A0C8091E8008B77809326
:101F9000E80031C0803879F58091E800877F809330
:101FA000E8008091ED018093F1008091E8008E7748
:101FB0008093E8000E94E00C1EC081111CC090912B
:101FC000F4019230C0F48091E800877F8093E800AC
:101FD0009093ED010E94E00C8091ED01811106C00B
:101FE0008091E30087FD02C081E001C084E080931E
:101FF000F1010E942A0A8091E80083FF0AC08091C3
:10200000E800877F8093E8008091EB0080628093F6
:10201000EB00AA960FB6F894DEBF0FBECDBFDF91DE
:10202000CF911F9108950895CF938091F101882356
:10203000A1F0C091E900CF709091EC00892F8170E0
:1020400090FD80E8C82B1092E9008091E80083FDA4
:102050000E94C20ECF70C093E900CF910895909373
:102060007501809374010895E0917401F0917501F8
:10207000309721F00190F081E02D099480E00895DF
:10208000E0917401F0917501309721F00280F381A5
:10209000E02D09940895E0917401F0917501309755
:1020A00021F00480F581E02D0994089520917201BA
:1020B000309173018217930771F0909373018093AD
:1020C0007201E0917401F0917501309721F0068062
:1020D000F781E02D099408952091700130917101EC
:1020E0008217930771F09093710180937001E091D2
:1020F0007401F0917501309721F00084F185E02D95
:102100000994089508950C9482100E94DC1B0E948B
:1021100035030C949E1C9F92AF92BF92CF92DF9298
:10212000EF92FF920F931F93CF93DF9300D000D0D5
:1021300000D0CDB7DEB70E944D030DE010E0AA2419
:10214000A394B12C902E802F0E943B049801295813
:102150003E4F6901F901F080F826A1F40150110900
:1021600088F78FEF89838A831B820E94E51B816039
:10217000782F9D838C8349815A816B818D810E9448
:1021800022112FC09091DA0191FF04C08E830E942A
:1021900041048E8125E030E0A501022E01C0440FEC
:1021A0000A94EAF7E42E4F21C1F029839A828E2106
:1021B00091E009F490E09B830E94E51B8160782FF9
:1021C0009D838C8349815A816B818D810E9422116C
:1021D000F6018081E826E08204C021503109E0F652
:1021E000BDCF0E94851F109176010E9434101817F0
:1021F000B9F00E9434108093760126960FB6F894B9
:10220000DEBF0FBECDBFDF91CF911F910F91FF9029
:10221000EF90DF90CF90BF90AF909F900C942D09DE
:1022200026960FB6F894DEBF0FBECDBFDF91CF91DB
:102230001F910F91FF90EF90DF90CF90BF90AF90E4
:102240009F900895CF93DF93CDB7DEB72B970FB64E
:10225000F894DEBF0FBECDBF4F83588769877A875A
:102260008B87DE01119686E0FD0111928A95E9F7D0
:1022700085E0FE01379601900D928A95E1F749813C
:102280005A816B817C818D819E810E946B172B9678
:102290000FB6F894DEBF0FBECDBFDF91CF9108958A
:1022A000CF93882309F4C2C0C82F823859F40E9402
:1022B000341081FDBBC089E30E94451A0E94121BA5
:1022C00089E30CC0833879F40E94341080FDAEC0DD
:1022D00083E50E94451A0E94121B83E50E94871A1B
:1022E000CF910C94121B843859F40E94341082FD53
:1022F0009DC087E40E94451A0E94121B87E4EECF1E
:102300008CEF8C0F813A48F48C2F0E94C8218111E8
:102310008DC08C2F0E94451AE3CF80E28C0F88304D
:1023200048F4C77081E001C0880FCA95EAF70E949F
:10233000CB1AD6CF8BE58C0F833078F4C53A29F0D1
:10234000C63A31F083E890E005C081E890E002C031
:1023500082E890E0CF910C94561088E58C0F833181
:1023600008F064C0C83A39F1C93A41F1CA3A49F1B2
:10237000CB3A51F1CC3A59F1CD3A61F1C03B69F118
:10238000CE3A71F1CF3A79F1C13B81F1C23B89F18B
:10239000C33B91F1C43B99F1C53BA1F1C63BA9F107
:1023A000C73BB1F1C83BB9F1C93BC1F1CA3BC9F167
:1023B00080E090E038C082EE90E035C089EE90E099
:1023C00032C08AEE90E02FC085EB90E02CC086EB07
:1023D00090E029C087EB90E026C08CEC90E023C011
:1023E0008DEC90E020C083E891E01DC08AE891E088
:1023F0001AC082E991E017C084E991E014C081E23B
:1024000092E011C083E292E00EC084E292E00BC041
:1024100085E292E008C086E292E005C087E292E0A1
:1024200002C08AE292E0CF910C946C10CF91089593
:10243000882309F44BC0823859F40E94341081FF7C
:1024400045C089E30E94451A0E94121B89E30CC013
:10245000833871F40E94341080FF38C083E50E94F5
:10246000451A0E94121B83E50E94871A0C94121BC6
:10247000843859F40E94341082FF28C087E40E94F7
:10248000451A0E94121B87E4EFCF9CEF980F913AF8
:1024900058F390E2980F983050F4877091E001C0A3
:1024A000990F8A95EAF7892F0E94D11ADFCF9BE511
:1024B000980F933020F480E090E00C945610885AE6
:1024C000833120F480E090E00C946C100895882310
:1024D00021F00E94CB1A0C94121B0895882321F03E
:1024E0000E94D11A0C94121B08957F928F929F9292
:1024F000AF92BF92CF92DF92EF92FF920F931F9312
:10250000CF93DF931F92CDB7DEB77C01C62E772E17
:10251000FC01058102950F70128111110E94E81AC9
:102520000E943E1A882379F0112369F080E28C0D15
:10253000883048F082E00E94271A0E943E1A91E0FB
:10254000D82ED92601C0D12CE72DE295EF70F0E00E
:10255000E05AFF4F0C94FD23872D807F072D0F70CD
:10256000882311F00295007F112389F0002309F4DC
:1025700090C180E28C0D883020F4802F0E94CB1A0D
:1025800003C0802F0E94DB1A0E94121B82C18C2D77
:102590000E941812002309F495C180E28C0D883046
:1025A00020F4802F0E94D11A03C0802F0E94E11ACC
:1025B0000E94121B87C1972D907F872D8F709032BC
:1025C00011F08295807FCC2021F0F1E0CF16B1F0A0
:1025D0001EC0112349F0002309F414C1013009F091
:1025E00011C10E94FB1A6EC1002319F0013009F4D9
:1025F00069C189830E94FE1A89810AC1112321F0D1
:10260000023008F05FC1FEC001115CC101C111239D
:1026100021F0002309F4F6C03CC1002309F4F8C0FE
:102620003EC1872D86958695837090E0009719F0BE
:10263000019761F047C1112321F08C2D972D9370E4
:1026400002C080E090E00E9456103CC1112321F0AE
:102650008C2D972D937002C080E090E00E946C104A
:1026600031C18C2D112319F00E948D1E02C00E94D1
:10267000F51E0E947A1F26C1872D837009F052C073
:10268000111120C18C2D829586958770880F880F37
:102690009C2D9F70892E912CA12CB12C082E04C04A
:1026A000880C991CAA1CBB1C0A94D2F7C4FE14C047
:1026B0000FE010E020E030E0B901A80104C0440FB1
:1026C000551F661F771F8A95D2F7CB01BA01609517
:1026D00070958095909503C060E070E0CB01272D48
:1026E00026952695237030E02230310569F023309D
:1026F000310589F0682979298A299B2921303105FA
:1027000071F00E94B318DEC0682979298A299B29B3
:102710000E94CF18D7C00E94B318C501B4010E940F
:102720009718D0C0112319F0872D817001C08695AC
:10273000882309F4C7C08C2D829586958770880FF1
:10274000880F9C2D9F70892E912CA12CB12C082EC6
:1027500004C0880C991CAA1CBB1C0A94D2F7C4FEA6
:1027600014C00FE010E020E030E0B901A80104C07F
:10277000440F551F661F771F8A95D2F7CB01BA0108
:10278000609570958095909503C060E070E0CB01F6
:10279000272D269526952370422F50E04230510573
:1027A00069F04330510589F0682979298A299B29E4
:1027B0004130510571F00E948D1984C06829792932
:1027C0008A299B290E94A9197DC00E948D19C501E3
:1027D000B4010E94711976C08C2D90E0FC01E05E7E
:1027E000F109E531F10508F050C0E059FF4F0C94B4
:1027F000FD230C2D0F70872D8F71112331F00E9456
:102800000A19802F0E9467125DC00E942B19802F29
:102810000E946E1257C0112339F0011153C0872D49
:102820008F710E9450194EC0023008F04BC0F7CF94
:10283000112339F0872D8F710E940A1943C011238B
:10284000C9F3872D8F710E942B193CC0112329F0E9
:10285000872D8F710E94F51835C00E94EB1832C089
:10286000112351F0172D1F71812F0E940A1963E067
:10287000812F0E941E1A26C081E00E94271A023072
:1028800008F182E00E94271A1DC0112331F00023B5
:1028900089F28C2D0E94501115C0002391F28C2DCD
:1028A0000E9418120FC0472D4F706C2DC7010E9457
:1028B00017050E940F1806C0472D4F706C2DC701D9
:1028C0000E943C06DD20F9F00E941A1A80FD1BC010
:1028D000F70112820E94141A0E940A19C7010E946D
:1028E00092140E94141A0F90DF91CF911F910F91B3
:1028F000FF90EF90DF90CF90BF90AF909F908F9020
:102900007F900C942B190F90DF91CF911F910F9115
:10291000FF90EF90DF90CF90BF90AF909F908F90FF
:102920007F9008950F931F93CF93DF93EC018881DD
:1029300099812B813C81232BB9F09F3F11F48F3F6C
:1029400099F0CE010E949405882371F06881798105
:102950008A810E94101A8C010E94C5190E948C184D
:10296000B801CE010E947512DF91CF911F910F9196
:1029700008950E94E81A0E94F81A0E94BD1A0E9447
:10298000121B0E942B200E947A1F80E090E00E9480
:10299000561080E090E00C946C100E94D81A0C94B1
:1029A000B9140E94051A292F22952F7030E02C307F
:1029B00031054CF42A3031056CF4225031092230B3
:1029C0003105A8F407C02C30310569F02F303105EE
:1029D00051F00DC0803F69F018F4803E40F409C00A
:1029E000843F29F406C093FB882780F9089580E08E
:1029F000089581E00895CF93DF9300D000D01F9217
:102A0000CDB7DEB70F900F900F900F900F90DF9122
:102A1000CF910895CF93DF9300D000D000D0CDB7F1
:102A2000DEB726960FB6F894DEBF0FBECDBFDF919E
:102A3000CF9108951F93CF93DF93C091850116E046
:102A400080918601C81799F0D0E01C9FF0011D9F6E
:102A5000F00D1124E957FE4F40815181628173814D
:102A6000848195810E940A152196C770E9CFDF9174
:102A7000CF911F9108954091B7015091B801609195
:102A8000B9017091BA018091BB019091BC010C9485
:102A90000A158091BC0182958F7009F054C0809115
:102AA000B901882309F44FC080918501A091860166
:102AB0006091B7017091B8014091BA015091BB018A
:102AC000B6E08A1709F43FC090E041155105C1F105
:102AD0007F3F11F46F3FA1F1B89FF001B99FF00D56
:102AE0001124E957FE4F218172132AC020816213FD
:102AF00027C02281211124C0238134812417350766
:102B000010F421503109241B350B283C3105C0F449
:102B10002091BC012F7020612093BC0126E0289FEA
:102B2000F001299FF00D1124E457FE4F80818F7032
:102B30008061808387EB91E00E9492140C941A15B7
:102B400001968770BECF0895CF92DF92EF92FF92E9
:102B50000F931F93CF93DF93CDB7DEB762970FB676
:102B6000F894DEBF0FBECDBF8C0185E0F801DE0119
:102B70001D9601900D928A95E1F7D8014C9111961E
:102B80005C91119712966C9112971396CD90DC90F0
:102B900014973091B7017091B8018091BA0190916A
:102BA000BB01009709F46BC17F3F19F43F3F09F463
:102BB00066C1E090B901EE2009F4C0C02091BC01CB
:102BC000C816D90628F0F601E81BF90BCF0104C09E
:102BD000809590958C0D9D1DFF24F394883C910564
:102BE00078F0F12C207F09F0C6C07C2DD98AC88AE4
:102BF00089890E94FB1487EB91E00E949214B1C076
:102C0000822F807F09F046C0751314C0341312C0A0
:102C1000611110C02F7020612093BC010E943B15F0
:102C200087EB91E00E9492148091BC01D801159627
:102C30008C932EC0CD2819F15F3F11F44F3FF9F06E
:102C4000F62E61111CC0809185012091860136E02D
:102C5000821709F45AC090E0389FF001399FF00DB7
:102C60001124E957FE4F7181571306C07081471335
:102C700003C07281711103C001968770E9CFF62EEF
:102C8000662309F418C18091BC0181608093BC0166
:102C9000F12C11C1751308C0341306C0611104C0B2
:102CA0008091BC01D801C3C04D875E878D859E850C
:102CB0006A8B0E94D1146A898823E1F16623D1F1DD
:102CC0002091BC01822F82958F7090E0029774F062
:102CD0008091B7019091B80198878F831986DB8620
:102CE000CA862C87CE0107960E94921486E0F801CE
:102CF000A7EBB1E001900D928A95E1F70E9449158A
:102D00000E943B15FF24F394D6C04D875E878D85C6
:102D10009E850E94051A292F22952F7030E02230BF
:102D200031050CF0BCC09F7009F0B6C0805E8830E1
:102D300008F4C1C0C8010E949214E4CFC816D90695
:102D400008F453C0F601E81BF90BCF01883C91054C
:102D500008F450C0F12C7C2DD98AC88A89890E9438
:102D6000FB14E7EBF1E086E0DF011D928A95E9F7BD
:102D70000E943B15A0C0751314C0341312C061111A
:102D800010C08091BC01F8018583C8010E94921493
:102D900086E0E7EBF1E0DF011D928A95E9F7FE2C72
:102DA0008AC04D875E878D859E856A8B0E94D1146F
:102DB0006A89882309F4BECF662309F4BBCF20912A
:102DC000BC01822F82958F7090E002970CF48ECF19
:102DD0008091B7019091B8019A8389831B82DD822B
:102DE000CC822E83CE0101967FCF809590958C0D5D
:102DF0009D1DACCFF62E662309F49CCF75132EC013
:102E000034132CC02091BC0120FD1FC0822F82955D
:102E10008F70D9F0D80115962C9315978F3049F003
:102E20008F5F982F9295907F822F8F70892B1596A8
:102E30008C93C8010E94921486E0F801A7EBB1E0E0
:102E400001900D928A95E1F793CF86E0F801A7EB08
:102E5000B1E001900D928A95E1F72DC04D875E8714
:102E60008D859E850E94D114811140CF8091BC0137
:102E700081608093BC01C8010E9492141CC066232B
:102E800009F458CF4D875E878D859E850E94D114A9
:102E9000882309F44FCF2ACF811148CF0CC02430AA
:102EA00031050CF047CF9F7009F440CFF8019581B0
:102EB000907F09F03BCF8F2D62960FB6F894DEBF5E
:102EC0000FBECDBFDF91CF911F910F91FF90EF907B
:102ED000DF90CF9008951F93CF93DF93CDB7DEB7E8
:102EE0002C970FB6F894DEBF0FBECDBF4F83588727
:102EF00069877A878B879C87CE0107960E94A415E5
:102F0000882369F08F8198852A853B85232BF1F1F1
:102F10009F3F09F063C08F3F09F060C037C086E073
:102F2000FE013796DE01119601900D928A95E1F728
:102F30006F817885EA85FB85309741F17F3F11F4F9
:102F40006F3F21F12091860130E0C9010196877021
:102F500099274091850150E08417950709F447C0EF
:102F600069837A83FD83EC8396E0929FD001939FDF
:102F7000B00D1124A957BE4FFE01319601900D925C
:102F80009A95E1F7809386010E941A1516E08091C8
:102F90008501909186018917C1F1189FC001112404
:102FA00089579E4F0E94A415882379F1E0918501ED
:102FB0001E9FF0011124E957FE4F4081518162812B
:102FC0007381848195810E940A158091850190E02A
:102FD00001968770992780938501D9CF4F815885B5
:102FE00069857A858B859C850E940A15CFCF0E94C2
:102FF000CD141092860110928501E7EBF1E086E096
:10300000DF011D928A95E9F7C1CF2C960FB6F8948F
:10301000DEBF0FBECDBFDF91CF911F910895EF921C
:10302000FF920F931F93CF93DF938C01009709F4C6
:103030006CC0F12CEE24E394E8012196F801849110
:10304000843740F4843008F051C0813081F0823000
:1030500019F15BC0853709F444C0A8F19CE7980FCB
:10306000903708F052C08F770E94181241C00E5F4F
:103070001F4FFE01C49180E28C0F883048F4C77066
:103080008E2D01C0880FCA95EAF70E94EB1A14C072
:103090008C2F0E9450112DC00E5F1F4FFE01C49156
:1030A00080E28C0F883058F4C7708E2D01C0880FD5
:1030B000CA95EAF70E94F11A0E94121B1AC08C2FBF
:1030C0000E94181216C00E5F1F4FFE01C491CC2340
:1030D00081F08FE99FE00197F1F700C00000C15037
:1030E000F6CF0E5F1F4FFE01F49003C00E945011F7
:1030F0008E018F2D882309F49FCFEFE9FFE03197F0
:10310000F1F700C000008150F5CFDF91CF911F9102
:103110000F91FF90EF90089508956093C10170930F
:10312000C2018093C3019093C4010C94B9140F930E
:103130001F930091C1011091C2012091C3013091F0
:10314000C401DC01CB01802B912BA22BB32B8093EC
:10315000C1019093C201A093C301B093C4011F9118
:103160000F910C94B9140F931F930091C10110910A
:10317000C2012091C3013091C401DC01CB01802345
:103180009123A223B3238093C1019093C201A09302
:10319000C301B093C4011F910F910C94B9140F9304
:1031A0001F930091C1011091C2012091C301309180
:1031B000C401DC01CB0180279127A227B32780938C
:1031C000C1019093C201A093C301B093C4011F91A8
:1031D0000F910C94B9141092BD011092BE0110927F
:1031E000BF011092C0010C94B91441E050E060E0BE
:1031F00070E004C0440F551F661F771F8A95D2F7F1
:103200004093BD015093BE016093BF017093C00114
:103210000C94B91441E050E060E070E004C0440F49
:10322000551F661F771F8A95D2F78091BD01909137
:10323000BE01A091BF01B091C001482B592B6A2B50
:103240007B2B4093BD015093BE016093BF017093EF
:10325000C0010C94B91441E050E060E070E004C09B
:10326000440F551F661F771F8A95D2F740955095DA
:10327000609570958091BD019091BE01A091BF01B4
:10328000B091C001482359236A237B234093BD0199
:103290005093BE016093BF017093C0010C94B914A8
:1032A00041E050E060E070E004C0440F551F661F2D
:1032B000771F8A95D2F78091BD019091BE01A091B0
:1032C000BF01B091C001482759276A277B27409347
:1032D000BD015093BE016093BF017093C0010C9477
:1032E000B9140F931F930091BD011091BE0120915D
:1032F000BF013091C001DC01CB01802B912BA22BAF
:10330000B32B8093BD019093BE01A093BF01B093F6
:10331000C0011F910F910C94B9140F931F9300914A
:10332000BD011091BE012091BF013091C001DC01AF
:10333000CB0180239123A223B3238093BD019093DB
:10334000BE01A093BF01B093C0011F910F910C94D7
:10335000B9140F931F930091BD011091BE012091EC
:10336000BF013091C001DC01CB0180279127A2274A
:10337000B3278093BD019093BE01A093BF01B0938A
:10338000C0011F910F910C94B9140895CF92DF9250
:10339000EF92FF920F931F93CF93DF938C01C09016
:1033A000C101D090C201E090C301F090C4018091AE
:1033B000BD019091BE01A091BF01B091C001C82A8A
:1033C000D92AEA2AFB2ACFE1D0E0D701C6010C2E88
:1033D00004C0B695A795979587950A94D2F780FF74
:1033E00006C0B8018C2F0E949208019721F4219702
:1033F00060F780E001C08C2FDF91CF911F910F917A
:10340000FF90EF90DF90CF900895CF93DF93EC0182
:103410000E94C619BE010E949208DF91CF910895C3
:10342000CB010E94051A08958091C5018595859567
:10343000859508958091C5018770089598E0899FCA
:1034400090011124262B2093C5010C940A19209178
:10345000C501809582238093C501982F977069F4E8
:1034600030E0482F552747FD50952417350729F0A0
:103470008595859585950C942B1908959091C50196
:10348000977081E009F480E0089590910C019923F0
:1034900021F090910D01911109C020910E01309100
:1034A0000F01F90132969FEF40E01FC0982F9695CB
:1034B000969596959F3050F5E0910E01F0910F0191
:1034C000E90FF11D877021E030E0A90102C0440F2F
:1034D000551F8A95E2F7CA019181892B818308954E
:1034E0009F3F39F04F5F4E3041F051915813F8CF64
:1034F0000DC05111F7CF942FF5CF9F3F39F0F9014F
:10350000E90FF11D97FDFA95828308950895909132
:103510000C01992321F090910D01911109C0209186
:103520000E0130910F01F9013296205F3F4F1FC00D
:10353000982F9695969596959F30F0F4E0910E0110
:10354000F0910F01E90FF11D877021E030E0A90132
:1035500002C0440F551F8A95E2F7CA0180959181F8
:103560008923818308953196E217F30729F090812A
:103570009813F9CF1082F7CF089581E090E0E091A1
:103580000E01F0910F01E80FF91F108201968031B2
:103590009105A9F708959091D901892B8093D901BC
:1035A000089580959091D90189238093D901089538
:1035B0001092D90108959091D801892B8093D80158
:1035C000089580959091D80189238093D80108951A
:1035D0001092D80108959091D701892B8093D7013B
:1035E000089580959091D70189238093D7010895FC
:1035F0001092D70108958093C60108951092C601D4
:10360000089580910E0190910F01FC0131969C016B
:10361000205F3F4F80E0919191118F5FE217F30798
:10362000D1F70895E0910E01F0910F018091D90139
:103630008083E0910E01F0910F0190818091D8017B
:10364000892B8083E0910E01F0910F019081809190
:10365000D701892B80838091C601882361F0E09196
:103660000E01F0910F019081892B80830E94011B34
:1036700081111092C60180910E0190910F010C945E
:10368000401020E0009739F0AC01415051098423EB
:1036900095232F5FF7CF822F0895CF92DF92EF927D
:1036A000FF926C01EE24FF24C114D104E104F10463
:1036B00021F0C701B60120E101C020E0C72ED82EBD
:1036C000E92EFF24C114D104E104F10419F0285FAC
:1036D000C701B6016B017C0154E0F694E794D794DE
:1036E000C7945A95D1F7C114D104E104F10419F03B
:1036F0002C5FC701B6016B017C0142E0F694E794B0
:10370000D794C7944A95D1F7C114D104E104F104C8
:1037100019F02E5FC701B601DC01CB01B695A79564
:1037200097958795892B8A2B8B2B09F02F5F822FFA
:10373000FF90EF90DF90CF9008958091F101843059
:1037400021F11092DB0120E488E190E00FB6F894BB
:10375000A895809360000FBE2093600080E00E94D7
:103760002D0983B7817F846083BF83B7816083BF66
:103770007894889583B78E7F83BF88E10FB6F894DD
:1037800080936000109260000FBE08950895089520
:103790000E94C61B0E944D030E94C71B0E94420448
:1037A00091E0811101C090E0892F08950E94CD140D
:1037B0000E9434100C942D0982E084BD93E095BDE5
:1037C0009AEF97BD80936E0008952FB7F89480917B
:1037D000DC019091DD01A091DE01B091DF012FBFEE
:1037E0000895CF92DF92EF92FF920F931F932FB71E
:1037F000F8944091DC015091DD016091DE017091FF
:10380000DF012FBF6A017B01EE24FF248C0120E041
:1038100030E0C016D106E206F30610F4415051091B
:103820009A01281B390BC9011F910F91FF90EF904E
:10383000DF90CF9008951F920F920FB60F92112430
:103840008F939F93AF93BF938091DC019091DD01A3
:10385000A091DE01B091DF010196A11DB11D809301
:10386000DC019093DD01A093DE01B093DF01BF91F5
:10387000AF919F918F910F900FBE0F901F90189551
:103880000E94310DF8942FEF87EA91E62150804095
:103890009040E1F700C0000087E090EBDC018093EE
:1038A000FB019093FC01A093FD01B093FE019CE00D
:1038B00088E10FB6F894A895809360000FBE9093AE
:1038C0006000FFCFEF92FF920F931F93CF93DF9390
:1038D000D82FCDE08C2F0E943B0405E010E0E82EAD
:1038E000F12CC701002E02C0959587950A94E2F746
:1038F00080FF09C0602F7C2F80E00E943D06D81316
:1039000002C081E006C00150110958F7C15010F7FC
:1039100080E0DF91CF911F910F91FF90EF9008957C
:10392000CF93C82F8CE20E94621C882321F08C2F39
:10393000CF910C94621C80E0CF910895CF930E94A8
:10394000E51D811102C00E94CB1DC5E6C15049F0A2
:103950000E944D038FE39CE90197F1F700C000003E
:10396000F5CF89E20E94901C811113C18AE20E9466
:10397000901C81110E94CB1D85E00E94901C81113A
:103980000E94401C0E94F01D8093DA0187E00E9493
:10399000901C8823A9F18BE10E94901C882351F090
:1039A0008091DA0181FB222720F991E0922790FB98
:1039B00081F90EC08EE00E94901C882361F08091F6
:1039C000DA0182FB222720F991E0922790FB82F90D
:1039D0008093DA0115C080E10E94901C9091DA0179
:1039E000882341F093FB222720F981E0822780FB86
:1039F00093F904C0892F809580FB90F99093DA01A8
:103A00008091DA010E94F41D0E94021E8093FA0147
:103A100080EE0E94901C882341F08091FA01982F3B
:103A2000909590FB80F98093FA0189E30E94901CA5
:103A3000882359F08091FA0181FB222720F991E037
:103A4000922790FB81F98093FA0182EE0E94901CEC
:103A5000882359F08091FA0182FB222720F991E016
:103A6000922790FB82F98093FA0186EE0E94901CC7
:103A7000882359F08091FA0183FB222720F991E0F5
:103A8000922790FB83F98093FA0183EE0E94901CA9
:103A9000882359F08091FA0184FB222720F991E0D4
:103AA000922790FB84F98093FA0185E30E94901C91
:103AB000882359F08091FA0185FB222720F991E0B3
:103AC000922790FB85F98093FA0181E30E94901C74
:103AD000882359F08091FA0186FB222720F991E092
:103AE000922790FB86F98093FA0181E10E94901C55
:103AF000882359F08091FA0187FB222720F991E071
:103B0000922790FB87F98093FA018091FA010E9435
:103B1000061E8091FA0187FB882780F980930D01AA
:103B200087E20E94901CC82F8EE10E94901C811198
:103B3000C2608FE10E94901C8111C46080E20E94EB
:103B4000901C8111C86081E20E94901C8111C061AB
:103B500082E20E94901C8111C06283E20E94901C4C
:103B60008111C06484E20E94901C882311F0C06817
:103B700002C0CC2329F08C2F0E94FD1D6C2F03C0A6
:103B80000E94F91D682F70E080E090E0CF910C94C6
:103B90008D18CF9108956DEE7EEF80E090E00E9449
:103BA000372460E082E090E00E94252460E083E01A
:103BB00090E00E94252460E084E090E00E942524AB
:103BC00060E085E090E00C94252480E090E00E9485
:103BD0001F2421E08D3E9E4F09F020E0822F0895A2
:103BE00082E090E00C941724682F82E090E00C941F
:103BF000252483E090E00C941724682F83E090E064
:103C00000C94252484E090E00C941724682F84E021
:103C100090E00C9425248091E20180FF0BC060911C
:103C2000130185E0689FB00111247595679575951E
:103C300067952BC081FF09C06091130185E0689FE3
:103C4000B00111247595679520C082FF07C060916F
:103C5000130185E0689FB001112417C09091E30122
:103C60009923D1F060911201961788F720911301E2
:103C700085E0289F90011124929FA001939F500DF1
:103C8000112470E0CA010E94E9236038710540F4F4
:103C90006115710539F002C065E070E0862F089566
:103CA0008FE7089581E008958091E20180FF08C0C8
:103CB0006091110170E0759567957595679521C0C4
:103CC00081FF06C06091110170E07595679519C07C
:103CD00082FF04C06091110170E010C09091E30177
:103CE0009923C1F0609110019617A0F780911101FE
:103CF000899FC001112470E00E94E923603871059A
:103D000028F46115710521F0862F08958FE7089535
:103D100081E0089561E070E0F4CF803F21F40E94DB
:103D20000B1E819504C0813F29F40E940B1E8093D5
:103D3000E6010895823F21F40E940B1E819504C084
:103D4000833F29F40E940B1E8093E5010895893F6B
:103D500019F40E94541E05C08A3F31F40E94541E7B
:103D600081958093E70108958B3F21F40E94541EB2
:103D7000819504C08C3F29F40E94541E8093E80171
:103D80000895843F21F48091E401816017C0853F4C
:103D900021F48091E401826011C0863F21F480917A
:103DA000E40184600BC0873F21F48091E4018860C6
:103DB00005C0883F31F48091E40180618093E40183
:103DC00008958D3F21F48091E20181600BC08E3F08
:103DD00021F48091E201826005C08F3F29F4809137
:103DE000E20184608093E2010895803F39F480917C
:103DF000E60187FF6CC01092E60169C0813F29F49B
:103E00008091E6011816BCF362C09091E501823FF3
:103E100029F497FF5CC01092E50159C0833F19F463
:103E20001916CCF354C0893F41F48091E70118166C
:103E30000CF04DC01092E7014AC08A3F29F48091EE
:103E4000E70187FF44C0F6CF8B3F39F48091E8014A
:103E500087FF3DC01092E8013AC08C3F29F4809161
:103E6000E8011816BCF333C0843F21F48091E401CB
:103E70008E7F17C0853F21F48091E4018D7F11C0B2
:103E8000863F21F48091E4018B7F0BC0873F21F4B2
:103E90008091E401877F05C0883F31F48091E4017F
:103EA0008F7E8093E40113C08D3F21F48091E20165
:103EB0008E7F0BC08E3F21F48091E2018D7F05C083
:103EC0008F3F29F48091E2018B7F8093E201809102
:103ED000E50181110EC08091E60181110AC0809137
:103EE000E701811106C08091E801811102C01092A2
:103EF000E301089584EE91E00E944B100E94E51BBF
:103F00009093E1018093E00108951F93CF93DF9395
:103F10008091E0019091E1010E94F11BAC01909130
:103F2000E301992321F02091140130E006C0209193
:103F300015018AE0289F900111244217530708F4C5
:103F400086C08091E501C091E601D091E701109112
:103F5000E801811107C0C11176C0D11174C01111DF
:103F600072C075C09F3F19F09F5F9093E3011816D0
:103F700024F40E940B1E8093E5018091E50187FFE8
:103F800005C00E940B1E81958093E5011C1624F448
:103F90000E940B1E8093E6018091E60187FF05C019
:103FA0000E940B1E81958093E6016091E5016623D6
:103FB00039F1C091E601CC2319F1772767FD70959F
:103FC000872F972F0E94FA2223E333E343E35FE333
:103FD0000E945E230E94C7226093E5016C2F772721
:103FE00067FD7095872F972F0E94FA2223E333E312
:103FF00043E35FE30E945E230E94C7226093E601D1
:104000001D1624F40E94541E8093E7018091E7015D
:1040100087FF05C00E94541E81958093E701111609
:1040200024F40E94541E8093E8018091E80187FFE8
:1040300005C00E94541E81958093E801DF91CF91C5
:104040001F910C947A1F9F3F09F08ECF96CFDF917E
:10405000CF911F910895E4EEF1E085E0DF011D921C
:104060008A95E9F71092E3011092E20108958330F6
:1040700081F128F4813059F08230D1F008958530F3
:1040800009F449C0B8F1863009F456C0089580910A
:104090001501262F30E0280F311D2F3F310524F464
:1040A000680F6093150108958FEF809315010895AF
:1040B00080911401262F30E0280F311D2F3F31054C
:1040C00024F4680F6093140108958FEF8093140116
:1040D000089580911301262F30E0280F311D2F3FC6
:1040E000310524F4680F6093130108958FEF8093D6
:1040F0001301089580911201262F30E0280F311D01
:104100002F3F310524F4680F6093120108958FEF5B
:1041100080931201089580911101262F30E0280F1D
:10412000311D2F3F310524F4680F6093110108956C
:104130008FEF80931101089580911001262F30E0B8
:10414000280F311D2F3F310524F4680F60931001B3
:1041500008958FEF809310010895833011F128F4B2
:10416000813049F0823091F00895853081F120F15D
:104170008630C1F1089580911501681720F4861BDF
:1041800080931501089510921501089580911401EE
:10419000681720F4861B809314010895109214016F
:1041A000089580911301681720F4861B80931301F2
:1041B000089510921301089580911201681720F458
:1041C000861B809312010895109212010895809128
:1041D0001101681720F4861B809311010895109235
:1041E0001101089580911001681720F4861B8093B7
:1041F000100108951092100108950F931F938D31AF
:1042000009F46BC008F03FC08E3009F47FC0C0F4E1
:10421000873009F469C068F4863009F0B1C0809134
:10422000DA01817F8E7F8093DA0181E08093EA0159
:10423000A8C0883009F4A2C08B3009F49FC0A0C088
:10424000863109F49BC078F4803109F472C0813161
:1042500009F096C00E94CD1490910D0181E089274C
:1042600080930D018BC0893109F488C08B3109F02E
:1042700087C08091DA0181FB222720F991E0922703
:1042800090FB81F94CC0853309F470C048F4873243
:1042900009F46CC008F459C0893209F467C070C0D1
:1042A000833438F48A3308F04EC0883309F466C08A
:1042B00067C0833409F45AC0883409F061C00E9491
:1042C000CD140FEF13ED20E3015010402040E1F733
:1042D00000C000000E94401C51C00E9481220E9428
:1042E00034100E942D094AC09091DA01892F8095DF
:1042F000817080FB90F929F0966098609093DA01C4
:1043000040C0997F977F9093DA0138C08091DA019D
:1043100082FB222720F991E0922790FB82F980937B
:10432000DA01992359F18091DA0181608093DA01F1
:1043300025C08091DA0183FB222720F991E09227A2
:1043400090FB83F9ECCF895301C08D5141E050E0DF
:1043500060E070E08A019B0104C0000F111F221F62
:10436000331F8A95D2F7C901B80104C061E070E03B
:1043700080E090E00E948D180E94CD1481E001C081
:1043800080E01F910F91089580E0089580E00895E6
:10439000CF93C82F8091EA01813079F018F08230F4
:1043A000E9F187C0E0910E01F0910F018081813128
:1043B00069F0823209F07FC009C0E0910E01F091EE
:1043C0000F018081813111F0823261F48C2F0E94C3
:1043D000C421811104C08C2F0E94FD201DC081E0EA
:1043E00090E01AC08C2F0E94C621811114C0C431E4
:1043F00079F048F4CB3079F0C03109F060C082E048
:104400008093EA0108C0C93219F0C83321F057C0BF
:104410001092EA0154C081E0817053C0C93289F121
:1044200018F5C43171F1A8F4C73009F046C08AE02C
:104430008093150194E19093140193E090931301FC
:104440008093120188E08093110188E2809310012B
:1044500034C0CE51C63088F5EC2FF0E0E65DFE4F5B
:1044600080818093E90129C0CE34E9F020F4CB3477
:1044700021F56AE013C0C13579F0C235F1F461E08D
:104480000DC08091E901882319F01092E90115C04F
:1044900081E08093EA0115C061E006C08091E901E6
:1044A0000E9437200AC06AE08091E9010E94AD2095
:1044B00004C01092EA0180E004C081E002C080E004
:1044C000ABCFCF910895E1E8F0E0808188608083F0
:1044D0008081816080838FB7F89493E09093890006
:1044E00090ED909388008FBF0895EFE6F0E0808113
:1044F000826080830895EFE6F0E080818D7F808385
:104500000895EFE6F0E0908182E0892780830895A6
:104510001F920F920FB60F9211242F933F934F9338
:104520005F936F937F938F939F93AF93BF93EF931B
:10453000FF938091EB019091EC0101969093EC0137
:104540008093EB01811103C082E00E942D09E0916C
:10455000EC01E695E695F0E0E854FB4FE49180919C
:10456000EB018E1303C080E00E942D09FF91EF91B3
:10457000BF91AF919F918F917F916F915F914F917B
:104580003F912F910F900FBE0F901F90189504D060
:104590006894B1118DC0089570D088F09F5790F045
:1045A000B92F9927B751A0F0D1F0660F771F881F58
:1045B000991F1AF0BA95C9F712C0B13081F077D0BF
:1045C000B1E0089574C0672F782F8827B85F39F05D
:1045D000B93FCCF3869577956795B395D9F73EF4B7
:1045E00090958095709561957F4F8F4F9F4F08955F
:1045F000E89409C097FB3EF490958095709561957D
:104600007F4F8F4F9F4F9923A9F0F92F96E9BB2732
:104610009395F695879577956795B795F111F8CFAE
:10462000FAF4BB0F11F460FF1BC06F5F7F4F8F4F19
:104630009F4F16C0882311F096E911C0772321F00F
:104640009EE8872F762F05C0662371F096E8862FA7
:1046500070E060E02AF09A95660F771F881FDAF7FE
:10466000880F9695879597F9089557FD9058440FB0
:10467000551F59F05F3F71F04795880F97FB991FC1
:1046800061F09F3F79F0879508951216130614067E
:10469000551FF2CF4695F1DF08C01616170618060B
:1046A000991FF1CF86957105610508940895E894E6
:1046B000BB2766277727CB0197F908950BD078C0E1
:1046C00069D028F06ED018F0952309F05AC05FC069
:1046D0001124EECFCADFA0F3959FD1F3950F50E0E0
:1046E000551F629FF001729FBB27F00DB11D639FA4
:1046F000AA27F00DB11DAA1F649F6627B00DA11D4A
:10470000661F829F2227B00DA11D621F739FB00DEF
:10471000A11D621F839FA00D611D221F749F33275F
:10472000A00D611D231F849F600D211D822F762FF8
:104730006A2F11249F5750408AF0E1F088234AF0F5
:10474000EE0FFF1FBB1F661F771F881F9150504041
:10475000A9F79E3F510570F014C0AACF5F3FECF35C
:10476000983EDCF3869577956795B795F795E7952D
:104770009F5FC1F7FE2B880F911D9695879597F93E
:10478000089597F99F6780E870E060E008959FEFD3
:1047900080EC089500240A941616170618060906D8
:1047A000089500240A9412161306140605060895A7
:1047B000092E0394000C11F4882352F0BB0F40F42F
:1047C000BF2B11F460FF04C06F5F7F4F8F4F9F4F6F
:1047D000089597FB072E16F4009407D077FD09D0B3
:1047E0000E94032407FC05D03EF4909581959F4FCD
:1047F0000895709561957F4F0895EE0FFF1F059006
:10480000F491E02D0994AA1BBB1B51E107C0AA1F1C
:10481000BB1FA617B70710F0A61BB70B881F991F61
:104820005A95A9F780959095BC01CD010895F99905
:10483000FECF92BD81BDF89A992780B50895A8E171
:10484000B0E042E050E00C943F24262FF999FECFCF
:1048500092BD81BDF89A019700B4021639F01FBAD3
:1048600020BD0FB6F894FA9AF99A0FBE08950196F2
:10487000272F0E9426240C942524DC01CB01FC0167
:10488000F999FECF06C0F2BDE1BDF89A319600B4A9
:0E4890000D9241505040B8F70895F894FFCFB4
:10489E0002202F09BD099A09660932090101C701D3
:1048AE0028080A03140A3F4D363979042C04F603FE
:1048BE00BD035003690382039B0301020304050633
:0448CE0007080900CE
:00000001FF
